:100000000C94BA050C94FE050C94FE050C94FE05A8
:100010000C94FE050C94FE050C94FE050C94FE0554
:100020000C94FE050C94FE050C945F1A0C94311B85
:100030000C9493280C94FE050C94FE050C94FE057C
:100040000C94FE050C94B1060C94FE050C94FE0570
:100050000C94FE050C94FB280C94FE050C94FE05F4
:100060000C94FE050C94FE050C94FE050C94FE0504
:100070000C94FE050C94FE050C94FE050C94FE05F4
:100080000C9445100C94FE050C94FE050C94FE0592
:100090000C94FE050C94FE050C94FE050C94FE05D4
:1000A0000C94FE050C94FE050C94FE0519072B0715
:1000B0003F07510759076F07BD07BD07BD07BD07BC
:1000C000BD07BD077D07AC079E1BC01BAE1CC01B38
:1000D000AE1C051C281CAE1C7D1C901C7A1F7A1FB0
:1000E000A91FA91FE81F08205E215E2113205E21A1
:1000F000C320C3202A2133215E215821D020D020C3
:10010000D020D020D020D020D020D020D020D0206F
:10011000D020D020D020D020D020D020E020EE2031
:10012000F520FC20062107634236B79BD8A71A3971
:10013000685618AEBAAB558C1D3CB7CC5763BD6D35
:10014000EDFD753EF6177231BF000000803F0800DC
:100150000000BE922449123EABAAAA2ABECDCCCC46
:100160004C3E00000080BEABAAAAAA3E00000000E0
:10017000BF000000803F0000000000084178D3BBB2
:100180004387D1133D190E3CC3BD4282AD2B3E685F
:10019000EC8276BED98FE1A93E4C80EFFFBE01C450
:1001A000FF7F3F0000000000000000000000000092
:1001B000000000010204060A0F17202C3A4A5D7164
:1001C000879DB3C7DAE9F5FCFFFCF5E9DAC7B39D13
:1001D00087715D4A3A2C20170F0A060402010000BD
:1001E00000000000000000006966207965730A09BC
:1001F0007065616E7574206275747465720A656CE1
:1002000073650A097269636520736E61636B7300BD
:10021000706C616E636B2F6578706572696D656E69
:1002200074616C20402076342E302D3230342D67AE
:100230003164316365642D6469727479002B001434
:10024000001A000800150017001C0018000C00120E
:100250000013002A00290004001600070009000A04
:10026000000B000D000E000F0033003400E1001DF4
:10027000001B0006001900050011001000360037B1
:1002800000380028000530E000E200E30003302CD5
:10029000002C0004305000510052004F002B00147D
:1002A000001A00090013000A000D000F0018001CBE
:1002B0000033002A0029000400150016001700076B
:1002C000000B00110008000C0012003400E1001DBA
:1002D000001B000600190005000E00100036003754
:1002E00000380028001450E000E200E30003302C46
:1002F000002C0004305000510052004F002B0034FD
:10030000003600370013001C0009000A0006001523
:10031000000F002A00290004001200080018000C39
:100320000007000B001700110016003800E1003331
:100330000014000D000E001B00050010001A00192B
:10034000001D0028000530E000E200E30003302C2F
:10035000002C0004305000510052004F0035021EA6
:10036000021F022002210222022302240225022669
:100370000227022A004C003A003B003C003D003EB0
:10038000003F002D022E022F0230023102010040F8
:100390000041004200430044004500320264020173
:1003A0000001000100010001000100010001000145
:1003B0000001000100AB00AA00A900AE0035001E3C
:1003C000001F002000210022002300240025002619
:1003D0000027002A004C003A003B003C003D003E54
:1003E000003F002D002E002F0030003100010040A2
:1003F0000041004200430044004500320032000149
:1004000000010001000100010001000100010001E4
:100410000001000100AB00AA00A900AE001E001EF2
:10042000001E001E001E001E001E001E001E001EDC
:10043000001E001E00000014001A0008001500171E
:10044000001C0018000C00120013002F0000000414
:10045000001600070009000A000B000D000E000F37
:1004600000330034000D30000000000600190000C9
:10047000000000110010000000000000000000005B
:10048000000000000000000000000000000000006C
:10049000000000000000000000000000000000005C
:1004A000000000000000000000000000000000004C
:1004B000000000000000000000000000000000003C
:1008300000000000000000000000000000010000B7
:100840005001000100010001000100010001000150
:100850000001004C00010001000100205021501354
:100860005012500030013002300C300100010027DE
:1008700050265023502450285029500100010001D7
:100880000001000100010001000100010001000160
:100890000001000100010001000100010000000052
:1008A00000000000002A2B280000000000000000CB
:1008B000000000000000000029000000002C1E3491
:1008C00020212224342627252E362D3738271E1F97
:1008D000202122232425263333362E37381F0405C2
:1008E000060708090A0B0C0D0E0F10111213141530
:1008F000161718191A1B1C1D2F3130232D3504050E
:10090000060708090A0B0C0D0E0F1011121314150F
:10091000161718191A1B1C1D2F3130354C000000FA
:1009200000000000000000000000000000000000C7
:1009300000000000000000000000000000000101B5
:10094000010101010001010101000000000000009F
:100950000000000000000001000100010101010190
:100960000101010101010101010101010101010177
:10097000010101010101010100000001010000006D
:100980000000000000000000000000000000000067
:1009900000000000000000000101010100280354D4
:1009A0000068006500200050006C0061006E00636C
:1009B000006B0020004B006500790062006F006151
:1009C000007200640000002C034F00720074006885
:1009D000006F006C0069006E00650061007200200D
:1009E000004B006500790062006F006100720064D6
:1009F00000730000000403090409026D00040100F3
:100A0000A0FA0904000001030101000921110100FD
:100A1000012240000705810308000A0904010001C2
:100A200003010200092111010001224D0007058286
:100A30000308000A09040200010300000009211153
:100A40000100012236000705830308000A09040398
:100A500000010300000009211101000122390007F3
:100A60000584031000011201100100000008EDFED2
:100A7000606001000102000105010906A1010507EE
:100A800019E029E71500250195087501810205087F
:100A900019012905950575019102950175039101CB
:100AA0000507190029771500250195787501810240
:100AB000C005010980A101850216010026B7001AB0
:100AC00001002AB700751095018100C0050C0901CD
:100AD000A1018503160100269C021A01002A9C022E
:100AE000751095018100C005010902A1010901A14C
:100AF00000050919012905150025019505750181D4
:100B0000029501750381010501093009311581251F
:100B10007F95027508810609381581257F95017535
:100B2000088106050C0A38021581257F9501750894
:100B30008106C0C005010906A101050719E029E7E2
:100B4000150025019508750181029501750881013F
:100B5000050819012905950575019102950175038F
:100B600091010507190029FF150026FF009506755C
:100B7000088100C011241FBECFEFDAE0DEBFCDBF79
:100B800004B603FE24C080918E0490918F04A0913E
:100B90009004B09191048730904BA740B04BB9F4CA
:100BA00010928E0410928F0410929004109291046F
:100BB00014BE84B7877F84BF88E10FB6F894809312
:100BC0006000109260000FBEE0E0F8E3099513E0CA
:100BD000A0E0B1E0EAE8F5E602C005900D92A0338E
:100BE000B107D9F714E0A0E3B3E001C01D92AE381D
:100BF000B107E1F70E94A9170C94C3320C940000CE
:100C000081E0089508950C9406080C9400060C9455
:100C100002060E948D2E811105C01092320310929F
:100C200031030DC081E290E00090330302C0880FD1
:100C3000991F0A94E2F7909332038093310382E084
:100C40008093300380916F00826080936F000895DD
:100C500090916F0081E0911101C080E008950E94A1
:100C60008D2E23E030E0281B3109220F209334031E
:100C70000895282F2F9880918000211108C0877F28
:100C80008093800010928D0010928C001BC08860B1
:100C900080938000233019F48FEF9FEF0FC083E023
:100CA00090E0821B9109880F991F2FEF3FEFA90158
:100CB00002C0569547958A95E2F7CA0190938D0038
:100CC00080938C000C942F06CF93C82F0E94280687
:100CD00040913303882329F090916F009D7F90937A
:100CE0006F00C09333038823D1F0209131033091FA
:100CF000320302C0369527954A95E2F72F733327C2
:100D0000C90102C0880F991FCA95E2F79093320378
:100D10008093310380916F00826080936F00CF9148
:100D200008950E942F0684E08093330310923003CD
:100D30000895279A2F988FEF9FEF909387008093C5
:100D400086008AE08093800089E1809381000E9480
:100D5000F62D0C9491060E9499066E9A769A0C9440
:100D6000DA071F920F920FB60F9211242F933F9321
:100D70008F939F93EF93FF93E0913103F0913203B0
:100D8000CF01019690933203809331030090330397
:100D900002C0F695E7950A94E2F7EF73809130036D
:100DA000823019F4E03251F404C0813039F4EF3369
:100DB00029F480916F008D7F80936F00F0E0E855FB
:100DC000FE4FE49121E031E0E29FC001E39F900DEE
:100DD00011240090340302C0969587950A94E2F797
:100DE00090938D0080938C00FF91EF919F918F9154
:100DF0003F912F910F900FBE0F901F901895CF939A
:100E0000DF93EC010E949429BE0180E090E0DF9125
:100E1000CF910C9489250F931F93462F50E04E30AD
:100E2000510508F0AAC0DC01FA01EA5AFF4F0C9400
:100E3000873212968C91882309F49FC000E010E05D
:100E4000980140E064E070E088E292E00E94C31301
:100E500081E090E011C012968C91882309F48DC036
:100E600000E010E0980140E066E070E088EB91E07F
:100E70000E94C31382E090E00E94FF067EC012969B
:100E80008C91882309F479C000E010E0980140E0DB
:100E900068E070E088EE91E00E94C31384E090E087
:100EA000EBCF12968C91882311F083E007C083E08A
:100EB00013C012968C91882371F084E00E9406265C
:100EC00082E00E9464060E94090640E164E083E03B
:100ED0000E94280E52C084E00E942726F6CF129668
:100EE0008C91882331F085EE0E941E1E0E944D2EAB
:100EF00044C085EE0E94E61E40C012968C91882365
:100F0000E1F10E94780F00E010E0980140E066E017
:100F100070E088E891E00E94C31384E00E942726D5
:100F200083E00E94272680E10E94272685E00E9418
:100F300006260E948129811102C00E945D290E941B
:100F4000992990E090938D0480938C04806880931D
:100F50008C040E949D2911C012968C91882369F0FF
:100F600000E010E0980140E066E070E088E591E084
:100F70000E94C31385E00E94272680E090E01F9125
:100F80000F9108950F931F932FEF89EF90E0215059
:100F900080409040E1F700C0000000E010E09801C0
:100FA00040E065E070E088E492E00E94C3131F9186
:100FB0000F9108950C94C2070F931F9300E010E067
:100FC000980140E063E070E080E091E00E94C3138C
:100FD0002FEF82E597E0215080409040E1F700C07C
:100FE00000001F910F910C94780F0F931F9300E056
:100FF00010E0980140E068E070E088E191E00E9434
:10100000C3131F910F9108950C94F507809140032D
:10101000882309F470C080913E0390913F030E94A1
:10102000D1288D3291400CF466C0109240030E948A
:1010300081088091380390913903499781F4809118
:101040003A0390913B03892B51F480913C0390919A
:101050003D03892B21F480E192E00E948208809177
:10106000380390913903099781F480913A03909164
:101070003B03892B51F480913C0390913D03892BD4
:1010800021F488EE91E00E948208809138039091CB
:101090003903049791F480913A0390913B0346976A
:1010A00061F480913C0390913D03892B31F48BE0F6
:1010B0000E941E1E8BE00E94E61E809138039091D4
:1010C00039030497C1F480913A0390913B0346970A
:1010D00091F480913C0390913D03079761F483EE76
:1010E0000E941E1E86E10E941E1E86E10E94E61ED0
:1010F00083EE0C94E61E089581E008950C947C081C
:10110000089508950F931F93CF938C01F8012491B4
:101110002223F9F030E0F901E356F74FC491F901C9
:10112000E35EF64F2491222359F081EE0E941E1EA9
:101130008C2F0E941E1E8C2F0E94E61E81EE04C082
:101140008C2F0E941E1E8C2F0E94E61E0F5F1F4FC9
:10115000DDCFCF911F910F9108950C94AB06809134
:101160008503882309F448C080914103909142038C
:10117000009779F40E94C52890934203809341031D
:101180008091430390E0009771F48091440390E0D4
:101190000AC00E94D1282091700230917102281754
:1011A000390740F329C00197880F991F880F991FAD
:1011B000FC01EB5BFC4F60817181828193810E9415
:1011C000AB0FE091430384E0E89FF0011124EB5B57
:1011D000FC4F60817181828193814FE050E00E94D9
:1011E00063138091430390E001966091440370E0A3
:1011F0000E947332809343030C940306109287037A
:101200000C94780F81E0809387030C940408089570
:101210008F929F92AF92BF92EF92FF920F931F9384
:10122000CF93DF93CDB7DEB7A3970FB6F894DEBFA9
:101230000FBECDBF7C01FC0100811181C8010E945D
:10124000C226B8010E940A0B8C01B7010E947E08D9
:10125000882309F4CCC10032F0E51F0741F4F701FF
:101260008281882309F458C00E945A14C0C10132F7
:10127000F0E51F0741F4F7018281882309F44CC08F
:101280000E946314B4C10232F0E51F0751F4F70164
:101290008281882309F440C00E9456148111F0CF46
:1012A000E3CF0332F0E51F0739F4F7018281882389
:1012B00099F10E9402099BC10432F0E51F0739F43D
:1012C000F7018281882341F10E94FE0890C1053216
:1012D000F0E51F0749F4F70182818823E9F0809146
:1012E00087038111F1CFE5CF0632F0E51F0739F40E
:1012F000F7018281882381F00E946A140AC00732B4
:10130000F0E51F0749F4F7018281882329F00E9444
:1013100075140E94F5076BC180918703811105C088
:10132000F70182818111CFC018C1003E110579F407
:10133000F7018281882309F44DC00E94780F81E073
:1013400080938603109285031092440350C1023E9D
:10135000110559F4F70182818823E1F10E94780F89
:10136000109286031092850342C1033E110591F449
:10137000F7018281882371F10E94780F1092860311
:1013800081E08093850310924303109242031092F0
:1013900041032DC10235110559F4F70182818823DB
:1013A00009F425C180917002909171020A970DC0D5
:1013B0000135110579F4F7018281882309F417C1F9
:1013C00080917002909171020A96909371028093BD
:1013D00070020DC14091740283E2EFE8F2E0DE0199
:1013E000119601900D928A95E1F7F701808121E035
:1013F00030E02C0F3D1F280F311DC90120917202D2
:1014000030917302FC01E20FF31F6081772767FDC3
:101410007095640F711D882777FD8095982F0E9425
:10142000952F20E030E040E451E40E94FA2E4B0179
:101430005C01F701218184E090E0821B9109BC01ED
:10144000882777FD8095982F0E94952F9B01AC01EE
:10145000C501B4010E94922E9B01AC0160E070E0D6
:1014600080E090E40E94083120E030E04CED50E450
:101470000E94A5304B015C01F70182818823D1F0E5
:101480004FE050E0C501B4010E94631380918603D0
:101490008823A1F08091440324E0829FF00111246D
:1014A000EB5BFC4F80829182A282B3828F5F80933C
:1014B000440304C0C501B4010E94AB0F0F3F1105E6
:1014C00008F02ECF94C08091400381111FC00431D9
:1014D00030E5130709F051C00E94800881E0809335
:1014E00040030E94C52890933F0380933E031092CF
:1014F0003703109239031092380310923B03109275
:101500003A0310923D0310923C0371C080913E0358
:1015100090913F030E94D128883C910570F48091FE
:101520003703E82FF0E0EE0FFF1FE85CFC4F11835C
:1015300000838F5F809337035AC0043880E5180713
:1015400021F00538104501F13AC0F7018281882366
:1015500041F01092350382E01EC0043830E51307D5
:1015600059F580913503811106C086E20E941E1E46
:1015700086E20E94E61E82E01CC00438F0E51F07E8
:1015800041F305381045D9F4F7018281882331F001
:101590001092360380E20E94351F29C080913603E5
:1015A000811106C087E20E941E1E87E20E94E61E8D
:1015B00080E20E943C1F1BC00538104529F381E0E2
:1015C0008093350380933603C701A3960FB6F89432
:1015D000DEBF0FBECDBFDF91CF911F910F91FF9066
:1015E000EF90BF90AF909F908F900C94050680E095
:1015F000A3960FB6F894DEBF0FBECDBFDF91CF919B
:101600001F910F91FF90EF90BF90AF909F908F90A0
:10161000089508959CE0799FF001112490E3899F3B
:10162000E00DF11D1124E60FF11DEE0FFF1FE35C2D
:10163000FD4F859194910895880F991FFC01E35403
:10164000FF4F859194910895880F991FFC01E35CE9
:10165000FD4F8591949108950F931F93CF93DF933E
:10166000EC01811521E39207A0F5C11580E3D807AD
:1016700008F0D7C0C83ED105D8F4C03ED10508F067
:1016800007C2C83AD10578F4C53AD10508F06AC056
:10169000C130D10509F463C008F4F7C1C430D105E5
:1016A00008F0F6C1F2C1CB3BD10508F466C0EDC12C
:1016B000C11590E2D90708F0AFC0C11521E0D207EB
:1016C00008F0E6C1C03FD10508F4DFC18E01106506
:1016D0001FC2C03880E5D80700F5C03790E5D907AC
:1016E00008F0A3C0C11520E5D20709F4ACC050F43E
:1016F000CE01905480319F4008F0C7C1DF708E0149
:10170000106A06C2C13080E5D80709F4AEC0C43102
:1017100090E5D90708F4AFC0B8C1C33820E5D207B7
:1017200009F48EC050F4C13890E5D90709F482C09D
:1017300008F083C000E011EDEBC1C03181E5D807AE
:1017400008F4A3C1C11597E5D90708F436C1CE0145
:1017500090578115904108F098C1DF7093C101E066
:1017600010E0D6C1C53AD10509F494C1C63AD105F5
:1017700009F093C102E810E4CBC1C83AD10509F4DD
:101780008FC1C93AD10509F48EC1CA3AD10509F40D
:101790008DC1CB3AD10509F48CC1CC3AD10509F4FD
:1017A0008BC1CD3AD10509F48AC1C03BD10509F4FA
:1017B00089C1CE3AD10509F488C1CF3AD10509F4DF
:1017C00087C1C13BD10509F486C1C23BD10509F4EB
:1017D00085C1C33BD10509F484C1C43BD10509F4DB
:1017E00083C1C53BD10509F482C1C63BD10509F4CB
:1017F00081C1C73BD10509F480C1C83BD10509F4BB
:101800007FC1C93BD10509F47EC1CA3BD10509F4AA
:101810007DC100E014E47CC1CE019F700E94240BC6
:1018200078C1DD278E01106C73C1CF70DD278E016A
:10183000146D6EC100E010ED6BC100E012ED68C1E7
:1018400000E013ED65C10E94C9210E94780F0E943B
:10185000DC078FEF94E32CE0815090402040E1F7CB
:1018600000C000000E94202953C180916204816061
:10187000809362044DC10E948129811102C00E949F
:101880005D290E94992990E090938D0480938C04A7
:10189000C23080E5D80721F480918C04816086C035
:1018A000C43090E5D90721F480918C0482607EC019
:1018B000C63020E5D20721F480918C04846076C084
:1018C000C83080E5D80719F480918C0427C0CA304D
:1018D00090E5D90721F480918C04806167C0CC30F9
:1018E00020E5D20721F480918C0480625FC0CE3065
:1018F00080E5D80721F480918C04806457C0C03102
:1019000090E5D90721F480918C0480684FC0C231E2
:1019100020E5D20729F480918C048460886046C059
:10192000C33080E5D80721F480918C048E7F3EC0BF
:10193000C53090E5D90721F480918C048D7F36C0A5
:10194000C73020E5D20721F480918C048B7F2EC014
:10195000C93080E5D80719F480918C0426C0CB30BB
:1019600090E5D90721F480918C048F7E1FC0CD3083
:1019700020E5D20721F480918C048F7D17C0CF30F1
:1019800080E5D80721F480918C048F7B0FC0C13192
:1019900090E5D90721F480918C048F7707C0C3317B
:1019A000D04531F480918C048B7F877F80938C04A9
:1019B00080918C040E949D29ABC08D2F99278F7038
:1019C000992781309105D9F49E012370332702C0F5
:1019D000880F991F2A95E2F79C688E0144E0000F5A
:1019E000111F4A95E1F700271370802B912B53E0CC
:1019F000CC0FDD1F5A95E1F7C076DD272FC082306E
:101A0000910531F4DC2FCC278E01016F106A80C064
:101A10008330910569F4CE018370992701E010E0CD
:101A200002C0000F111F8A95E2F7C8019C680FC021
:101A300084309105B9F4CE018370992701E010E05C
:101A400002C0000F111F8A95E2F7C8019A6823E0CF
:101A5000CC0FDD1F2A95E1F7C07ED7708C010C2BCF
:101A60001D2B56C08530910531F4DC2FCC278E011B
:101A7000046F106A4DC0069709F04AC0CF71DD2788
:101A8000DC2FCC278E01106243C000E010E040C084
:101A90008E013EC001E810E43BC003E810E438C00A
:101AA00002EE14E435C009EE14E432C00AEE14E488
:101AB0002FC005EB14E42CC006EB14E429C007EB9F
:101AC00014E426C00CEC14E423C00DEC14E420C094
:101AD00003E815E41DC00AE815E41AC002E915E49C
:101AE00017C004E915E414C001E216E411C003E2D2
:101AF00016E40EC004E216E40BC005E216E408C0CA
:101B000006E216E405C007E216E402C00AE216E4A3
:101B1000C801DF91CF911F910F9108959CE0799FAB
:101B2000F001112490E3899FE00DF11D1124E60FCF
:101B3000F11DEE0FFF1FE35CFD4F85919491803EF8
:101B40009105E0F4803C910558F58133910509F445
:101B50006FC048F48932910509F463C08A32910557
:101B600009F46DC072C089339105E9F0823891059E
:101B7000D1F08533910509F44DC067C0833E9105CE
:101B800081F138F4803E9105B9F0823E9105D9F09B
:101B90005CC0863E910561F1873E9105A1F155C07B
:101BA0000E941C0B089520918C0420FD02C021FF8F
:101BB0004CC080EE90E049C080918C0480FFF9CF4A
:101BC00089E390E042C080918C0482FF0EC0809136
:101BD0008C0484FF03C080E090E037C083EE90E087
:101BE00034C080918C0482FFF2CF82EE90E02DC051
:101BF00080918C0483FF0BC080918C0484FDEBCF1B
:101C000087EE90E022C080918C0483FFF5CF86EEB2
:101C100090E01BC080918C0485FF07C089E290E0B2
:101C200014C080918C0485FFF9CF85E390E00DC04E
:101C300080918C0486FF07C08AE290E006C0809104
:101C40008C0486FFF9CF81E390E00E942C0B08956D
:101C5000CF92DF92EF92FF920F931F9301E010E07B
:101C600020E030E06801790104C0CC0CDD1CEE1CE2
:101C7000FF1C8A95D2F704C0000F111F221F331FCB
:101C80006A95D2F70C291D292E293F29C0904504B9
:101C9000D0904604E0904704F0904804C022D1223E
:101CA000E222F322842FC016D106E206F30641F4A5
:101CB0001F910F91FF90EF90DF90CF900C9406262C
:101CC0001F910F91FF90EF90DF90CF900C942726FB
:101CD0000C940706E82FF0E0E254FD4F8081E82FD6
:101CE000EF70F0E082958F7021E030E0A90102C032
:101CF000440F551F8A95E2F740A308950F931F9351
:101D0000CF93DF9385B7806885BF85B7806885BF2F
:101D1000C3E0D0E001E010E0FE01E254FD4F80811D
:101D2000E82FEF70F0E021A182958F70A80102C02A
:101D3000440F551F8A95E2F7CA01822B81A38C2F8D
:101D40000E946A0E219740F78BE090E061E070E01E
:101D5000FC01EE54FD4F2081E22FEF70F0E042A134
:101D600022952F70DB0102C0AA0FBB1F2A95E2F754
:101D70009D01242B22A3019758F7DF91CF911F914A
:101D80000F910C94AD08EF92FF920F931F93CF9396
:101D9000DF9300E913E0C3E0EE24E394F12CD5E0F7
:101DA0008C2F0E946A0E8BE090E040E050E0FC0136
:101DB000EE54FD4F6081E62FEF70F0E020A130E09F
:101DC00062956F7002C0359527956A95E2F720FD00
:101DD00009C09701082E02C0220F331F0A94E2F7B0
:101DE000422B532B019718F7F801929182918F01A2
:101DF0008417950721F051834083D09375028C2F6F
:101E00000E946A0EC15060F68091750287FD2CC059
:101E10008150809375028F3F39F08FE99FE00197E1
:101E2000F1F700C0000020C080918E0390918F03D5
:101E3000909397038093960380918C0390918D03E8
:101E4000909395038093940380918A0390918B03E0
:101E500090939303809392038091880390918903D8
:101E600090939103809390030E94AF0881E0DF91EB
:101E7000CF911F910F91FF90EF900895E82FF0E020
:101E8000EE0FFF1FE057FC4F808191810895089568
:101E90000F931F93CF9308E913E0C0E0F8019291EC
:101EA00082918F010E943D28C80FF3E000391F077F
:101EB000A9F78C2FCF911F910F9108950E9481292E
:101EC000811102C00E945D290E94AB298093770492
:101ED0003E9A809171008D7F8093710082E08093A3
:101EE00090008AE18093910081E080939A030895A5
:101EF00080919A03811102C00E945E0F1092EA0342
:101F00001092E903809171008D7F80937100809120
:101F100090008F73809390001092AC031092AB03EB
:101F20001092E3031092E4031092E5031092E6038B
:101F30001092E2031092E103E1ECF3E0A1EBB3E0D5
:101F400011921192119211921D921D9283E0E13E25
:101F5000F807B1F70895CF92DF92EF92FF920F93B7
:101F60001F93CF93DF932091AB03222309F484C006
:101F70006B017C0180919A03811102C00E945E0F67
:101F800001EE13E0C7E0D0E0A7019601F8019291BD
:101F90008291729162918F010E94F62E811131C05F
:101FA000FE01EE0FFF1FEE0FFF1FEF53FC4F1082DD
:101FB000118212821382DE01AA0FBB1FAF54BC4FE5
:101FC00011961C921E92C730D105E9F021964481EA
:101FD0005581668177814083518362837383148244
:101FE00015821682178212968D919C9113971196E5
:101FF0009C938E9313961C921E921297349612966F
:10200000E2CF219708F68091E9039091EA030197C6
:1020100097FD05C09093EA038093E90304C01092F2
:10202000EA031092E9038091E9039091EA03209179
:10203000E7033091E8032817390724F01092E803EA
:102040001092E703892BC1F4809171008D7F8093FA
:102050007100809190008F73809390001092E30341
:102060001092E4031092E5031092E6031092E2034B
:102070001092E1031092AB03DF91CF911F910F916A
:10208000FF90EF90DF90CF9008951F920F920FB6C0
:102090000F9211244F925F926F927F928F929F9234
:1020A000AF92BF92CF92DF92EF92FF922F933F9326
:1020B0004F935F936F937F938F939F93AF93BF9350
:1020C000CF93DF93EF93FF938091AB03882309F4C1
:1020D0009BC1C091E903D091EA031C161D060CF0C8
:1020E00093C140909B0350909C0360909D0370901F
:1020F0009E0320E030E0A901C301B2010E94A1309B
:1021000018160CF065C0C130D10509F452C0809199
:10211000E7039091E803BE010E9473327C01909323
:10212000E8038093E7038090AD039090AE03A09006
:10213000AF03B090B00320E030E040E85FE3C501BA
:10214000B4010E94922E6093AD037093AE0380930E
:10215000AF039093B003F701EE0FFF1FEE0FFF1FC9
:10216000EF53FC4FA30192016081718182819381C1
:102170000E94FA2E20E030E040E05EE30E94A530AD
:102180009B01AC01C501B4010E94A13018168CF46A
:10219000C7010196BE010E9473329093E8038093B9
:1021A000E7031092AD031092AE031092AF031092AA
:1021B000B003E091E703F091E803EE0FFF1FEE0F8D
:1021C000FF1FEF53FC4F6081718182819381D0C0EA
:1021D000C090E303D090E403E090E503F090E603C1
:1021E00020E030E0A901C701B6010E94F62E219738
:1021F000882309F4A2C0FE01EE0FFF1FEE0FFF1FA0
:10220000EF53FC4F80809180A280B380A5019401A0
:10221000C701B6010E94F62E87FF31C0A5019401C7
:1022200060E070E08CED93EC0E94FA2E20E030E04C
:1022300040E451E40E94FA2E20E030E040E05FE309
:102240000E94A5309B01AC0160E070E080E090E46A
:102250000E9408319B01AC01C501B4010E94A53068
:102260009B01AC01C701B6010E94F62E87FF07C093
:10227000A701960160E070E08CED93E439C0A50100
:102280009401C701B6010E94A13018160CF055C088
:10229000A501940160E070E08CED93E40E94FA2EB9
:1022A00020E030E040E451E40E94FA2E20E030E0EB
:1022B00040E05FE30E94A5309B01AC0160E070E06C
:1022C00080E090E40E9408319B01AC01C501B4019B
:1022D0000E94A5309B01AC01C701B6010E94A1304C
:1022E00018165CF5A701960160E070E08CED93ECA8
:1022F0000E94FA2E20E030E040E451E40E94FA2EE1
:1023000020E030E040E05FE30E94A5309B01AC019B
:1023100060E070E080E090E40E9408319B01AC0135
:10232000C701B6010E94A5306093E3037093E403F4
:102330008093E5039093E60313C0FE01EE0FFF1FA9
:10234000EE0FFF1FEF53FC4F80819181A281B3817B
:102350008093E3039093E403A093E503B093E60333
:102360006091E3037091E4038091E5039091E603AB
:1023700020919803309199032F3F4FEF340731F0AC
:102380002F5F3F4F30939903209398030E9480144E
:102390006B017C0120E034E244EF51E40E94F62E10
:1023A00087FF08C086EFC82E88E2D82E84EFE82E7B
:1023B00081E4F82E20E030E040E051E4C701B601AE
:1023C0000E94A5309B01AC0160E074E284E79BE4CD
:1023D0000E94FA2E6B017C010E94672F7093970078
:1023E00060939600209176023091770240917802B6
:1023F00050917902C701B6010E94A5300E94672F53
:1024000070939900609398008091AC03882309F43D
:1024100033C1C090A703D090A803E090A903F09027
:10242000AA0320E030E0A901C701B6010E94A13053
:102430001816D4F580919803909199038F3F2FEF50
:10244000920729F001969093990380939803C7010E
:10245000B6010E94801420E030E040E051E40E9488
:10246000A5309B01AC0160E074E284E79BE40E942C
:10247000FA2E6B017C010E94672F70939700609386
:102480009600209176023091770240917802509127
:102490007902C701B6010E94A5300E94672F709390
:1024A00099006093980008C01092970010929600CF
:1024B00010929900109298006091A1037091A2036C
:1024C0006F5F7F4F7093A2036093A10320919600EA
:1024D0003091970080E090E0232BF1F0C0919600BE
:1024E000D09197000E94932F6B017C01BE0180E088
:1024F00090E00E94932F9B01AC016091A303709127
:10250000A4038091A5039091A6030E94FA2E20E0D7
:102510003FEF4FE757E410C00E94932F6B017C01FF
:1025200020E030EE4FEF54E46091A3037091A403D8
:102530008091A5039091A6030E94A5309B01AC0158
:10254000C701B6010E94A13087FD96C080919F030C
:102550008F5F80939F0390E0209173043091740407
:1025600082179307A0F080917E04882319F01092BF
:102570009F030DC0809171008D7F809371008091C9
:1025800090008F73809390001092AC037DC0809177
:10259000A003C0919F03811128C0C0907804D090FF
:1025A0007904E0907A04F0907B0420E030E0A90107
:1025B000C701B6010E94A1301816BCF481E08093D7
:1025C000A0031092A7031092A8031092A9031092DF
:1025D000AA03C092A303D092A403E092A503F092B1
:1025E000A603C150C0939F0343C01092A003109252
:1025F000990310929803E0917504F091760448E0F5
:10260000C49FE00DF11D112480819181A281B381CD
:102610008093A7039093A803A093A903B093AA0360
:1026200020E030E040E85EE3648175818681978137
:102630000E94A5306B017C0180917A02682F70E0C6
:1026400080E090E00E94932F20E030E048EC52E4DC
:102650000E94FA2E9B01AC01C701B6010E94A53071
:102660006093A3037093A4038093A5039093A603A0
:102670001092A2031092A1038091770480FD04C000
:102680001092AC031092AB03FF91EF91DF91CF91C9
:10269000BF91AF919F918F917F916F915F914F917A
:1026A0003F912F91FF90EF90DF90CF90BF90AF9030
:1026B0009F908F907F906F905F904F900F900FBE84
:1026C0000F901F901895CF92DF92EF92FF92CF93C9
:1026D000DF936B017C01EA0180919A03811102C0B2
:1026E0000E945E0F8091770480FF46C08091E903CD
:1026F0009091EA0308970CF03FC0809171008D7FA4
:10270000809371008091AC0381110E94780F81E069
:102710008093AB03109299031092980320E030E06D
:10272000A901C701B6010E94A1301816DCF48091FE
:10273000E9039091EA03FC01EE0FFF1FEE0FFF1F6C
:10274000EF53FC4FC082D182E282F382FC01EE0F94
:10275000FF1FEF54FC4FD183C08301969093EA038F
:102760008093E90380917100826080937100809171
:102770009000806880939000DF91CF91FF90EF9060
:10278000DF90CF9008958F929F92AF92BF92CF9299
:10279000DF92EF92FF920F931F93CF93DF93EC01A1
:1027A0007B01D42E4801590180919A03811102C006
:1027B0000E945E0F8091770480FF6BC08091710052
:1027C0008D7F809371008091AB0381110E94780FFF
:1027D00081E08093AC03D0937604C0937504F092AB
:1027E0007404E0927304D0927E04809278049092F4
:1027F0007904A0927A04B0927B041092AD031092F7
:10280000AE031092AF031092B00310929F03888121
:102810009981AA81BB818093A7039093A803A09379
:10282000A903B093AA0320E030E040E85EE36C81A6
:102830007D818E819F810E94A5306B017C018091FA
:102840007A02682F70E080E090E00E94932F20E0F1
:1028500030E048EC52E40E94FA2E9B01AC01C70123
:10286000B6010E94A5306093A3037093A4038093E4
:10287000A5039093A6031092A2031092A103809146
:1028800071008260809371008091900080688093D5
:102890009000DF91CF911F910F91FF90EF90DF900B
:1028A000CF90BF90AF909F908F90089580917704C4
:1028B00081700895809177048160809377040E94ED
:1028C000AF290C940709809177048E7F8093770459
:1028D0000C94AF298091EB0390E0019666E070E0E4
:1028E0000E9473328093EB0308958091EB0390E094
:1028F000019766E070E00E9473328093EB030895C5
:102900008F929F92AF92BF92CF92DF92EF92FF92FF
:102910000F931F93CF93DF936B017C01C0919803BA
:10292000D0919903BE0180E090E00E94932F4B016B
:102930005C01A701960160E070E08CE594E40E94E0
:10294000FA2E9B01AC01C501B4010E94A5300E9482
:10295000672F2091EB03233009F473C028F422235E
:1029600051F02130E9F02CC1243009F4A0C0253009
:1029700009F4E0C025C180E090E0A0E0BFE38093CF
:10298000760290937702A0937802B0937902109226
:102990009B0310929C0310929D0310929E0310C102
:1029A00010929B0310929C0310929D0310929E0321
:1029B0006431710540F46A30710560F520E030E063
:1029C00040E85EE32BC0693C710508F0AAC080E0D6
:1029D00090E00E94932F20E030E040EA51E40E9412
:1029E000912E20E030E044E353E40E94FA2E9B0154
:1029F000AC010E94A53020E030E040E05EE30E94A0
:102A0000A5309B01AC0160E070E080E09EE30E9495
:102A1000912E44C020E030E040E05FE3C701B60102
:102A20000E94A5306B017C0180E090E0A0E0BEE355
:102A30008093760290937702A0937802B093790204
:102A4000BFC010929B0310929C0310929D031092A2
:102A50009E034AE0469F9001479F300D1124C90113
:102A600068EB7BE00E945F32BC016C5D754077FFD4
:102A700003C0719561957109882777FD8095982F1E
:102A80000E94952F2EE333EC4EE259E30E94A530CD
:102A900020E030E040EC5EE30E94922E60937602EC
:102AA00070937702809378029093790289C0109294
:102AB0009B0310929C0310929D0310929E03CE01E3
:102AC00083709927892BE1F0BE016170772780E040
:102AD00090E00E94932F20E030E040E05EE30E940F
:102AE000A53020E030E040E45FE30E94922E609346
:102AF00076027093770280937802909379020CC0EB
:102B000080E090E0A0E0BFE38093760290937702AC
:102B1000A0937802B0937902C770DD27CD2B09F01E
:102B20004FC01092760210927702109278021092A3
:102B3000790246C010929B0310929C0310929D0351
:102B400010929E0300E010E020E03FE30093760245
:102B500010937702209378023093790267397105D8
:102B600078F180E090E00E94932F20E030E047E190
:102B700053E40E94912E20E030E04AE754E40E94A2
:102B8000FA2E20E030E048E452E40E94A53020E034
:102B900030E040EA51E40E94D72F0E94622F660F76
:102BA000771F660F771FFB01EE53FD4F20813181A8
:102BB00042815381C701B6010E94A5306B017C019F
:102BC000C701B601DF91CF911F910F91FF90EF9058
:102BD000DF90CF90BF90AF909F908F90089580919D
:102BE000FC030895CF93DF9300D01F92CDB7DEB7DB
:102BF0009C0180918304843019F593E099833B8391
:102C00002A839093E9008FEF9091E800815095FD21
:102C100006C095ED9A95F1F700008111F5CF8091EE
:102C2000E80085FF0DC040E050E063E070E0CE01B9
:102C300001960E944F188091E8008E778093E800FB
:102C40000F900F900F90DF91CF910895CF93DF9366
:102C500000D01F92CDB7DEB720918304243021F538
:102C600022E029839B838A8383E08093E9008FEFAE
:102C70009091E800815095FD06C095ED9A95F1F789
:102C800000008111F5CF8091E80085FF0DC040E084
:102C900050E063E070E0CE0101960E944F188091F1
:102CA000E8008E778093E8000F900F900F90DF91EF
:102CB000CF910895209183042430F1F422E02093F1
:102CC000E9002FEF3091E800215035FD06C035EDC9
:102CD0003A95F1F700002111F5CF2091E80025FF8A
:102CE0000BC040E050E065E070E00E944F1880911A
:102CF000E8008E778093E8000895CF93DF93EC018E
:102D000090918304943009F046C080918502882315
:102D1000D9F0809186028823B9F09093E9008FEF73
:102D20009091E800815095FD06C095E19A95F1F7E4
:102D300000008111F5CF8091E80085FF2CC040E0B4
:102D400050E060E170E017C081E08093E9008FEF10
:102D50009091E800815095FD06C095ED9A95F1F7A8
:102D600000008111F5CF8091E80085FF14C040E09C
:102D700050E068E070E0CE010E944F188091E800BA
:102D80008E778093E80080E1FE01ACEEB3E0019025
:102D90000D928A95E1F7DF91CF9108958091820499
:102DA000811109C00E94E4190E94411A8091E20039
:102DB00084608093E200089510928204089508953B
:102DC00008950C94882842E061EC81E00E945E192D
:102DD00042E061EC82E00E945E1942E061EC83E037
:102DE0000E945E1942E161EC84E00C945E198091CE
:102DF0008504833009F455C030F4813071F082309D
:102E000009F48EC008958A3009F47AC08B3009F431
:102E100060C0893009F09CC020C080918404813A50
:102E200009F096C08091E800877F8093E800809148
:102E3000880490918904892B21F460E18CEE93E061
:102E400003C060E080E090E070E00E949A188091FA
:102E5000E8008B778093E8000895809184048132A4
:102E600009F076C08091880490918904009719F048
:102E7000039709F06DC08091E800877F8093E80098
:102E80008091E80082FD05C0809183048111F8CF14
:102E90005FC08091F1008093FC038091E8008B7704
:102EA00053C080918404813A09F052C08091880413
:102EB00090918904892B09F04BC08091E800877FAD
:102EC0008093E8008091E80080FFFCCF809185022C
:102ED00036C0809184048132D9F580918804909124
:102EE0008904892BA9F58091E800877F8093E80009
:102EF0000E94931980918604809385020C94C921C5
:102F000080918404813221F58091E800877F80934D
:102F1000E8000E949319809187048093FD0308952F
:102F200080918404813AA1F48091E800877F8093A6
:102F3000E8008091E80080FFFCCF8091FD03809342
:102F4000F1008091E8008E778093E8000C9493194B
:102F5000089584B7877F84BF88E10FB6F894809383
:102F60006000109260000FBE80E8809361001092B4
:102F700061000E94361D0E94E4190E94411A80914E
:102F8000E20084608093E20078940E94C71C0E9453
:102F9000381D8BE792E00E94E21C8091830485300B
:102FA00069F40E944928809181048823B1F30E942A
:102FB0007728882391F30E943918EFCF0E94401D93
:102FC000ECCF292F332723303105C9F064F42130A9
:102FD000310581F02230310509F043C08DE690E0E3
:102FE00029EF39E042C021323105F1F022323105BA
:102FF00041F137C082E190E026E63AE036C09927F9
:103000008130910541F08230910541F0892B49F5DD
:10301000E5EFF9E005C0E7ECF9E002C0EDE9F9E021
:10302000849190E09F0121C06430D8F4E62FF0E055
:10303000EE0FFF1FE25EFC4F2081318189E090E0BE
:1030400014C0643070F470E0FB01EE0FFF1FEA5E05
:10305000FC4F20813181FB01EE5EFC4F808190E0CE
:1030600004C080E090E020E030E0FA01318320836A
:10307000089580E189BD82E189BD09B400FEFDCFDC
:103080008091D8008F7D8093D8008091E00082608D
:103090008093E0008091E00081FDFCCF0895CF9205
:1030A000DF92EF92FF920F931F93CF93DF93EC0188
:1030B0008B016A010E94B219811133C0C114D1047D
:1030C00039F0F60180819181081B190BC80FD91FB7
:1030D000E12CF12C0115110519F18091E80085FD15
:1030E00016C08091E8008E778093E800C114D10467
:1030F00049F0F60180819181E80EF91EF182E082AB
:1031000085E00FC00E94B219882321F30AC089917B
:103110008093F10001501109FFEFEF1AFF0ADACF97
:1031200080E0DF91CF911F910F91FF90EF90DF90A2
:10313000CF90089520918A0430918B042617370789
:1031400048F06115710539F42091E8002E7720933D
:10315000E80001C0B90140E061157105A9F12091B5
:103160008304222309F443C0253009F442C020918E
:10317000E80023FD40C02091E80022FD32C02091EC
:10318000E80020FFE9CF4091F3002091F20030E009
:10319000342BFC01CF016115710559F02830310540
:1031A00040F481918093F100615071092F5F3F4F8E
:1031B000F1CF41E02830310509F040E02091E800EE
:1031C0002E772093E800C8CF4111C9CF0AC0809163
:1031D0008304882361F0853061F08091E80083FDED
:1031E0000AC08091E80082FFF2CF80E0089582E07B
:1031F000089583E0089581E0089520918A04309134
:103200008B042617370748F06115710539F42091B2
:10321000E8002E772093E80001C0B901FC0120E00E
:103220006115710591F180918304882309F440C0F0
:10323000853009F43FC08091E80083FD3DC0809156
:10324000E80082FD2FC08091E80080FFE9CF209147
:10325000F3008091F20090E0922B6115710559F016
:103260008830910540F424912093F100319661500B
:1032700071090196F2CF21E0089709F020E08091D2
:10328000E8008E778093E800CBCF2111CCCF0AC025
:1032900080918304882361F0853061F08091E8009B
:1032A00083FD0AC08091E80082FFF2CF80E008959C
:1032B00082E0089583E0089581E00895982F973083
:1032C00058F59093E900981739F07091EC0020912F
:1032D000ED005091F00003C0242F762F50E021FF25
:1032E00019C03091EB003E7F3093EB003091ED0040
:1032F0003D7F3093ED003091EB0031603093EB0077
:103300007093EC002093ED005093F0002091EE00BC
:1033100027FF07C09F5FD3CF8F708093E90081E0C4
:10332000089580E008958091840487FF11C0809102
:10333000E80082FD05C0809183048111F8CF11C09F
:103340008091E8008B770BC080918304882349F03B
:103350008091E80080FFF8CF8091E8008E7780931D
:10336000E80008952091E4003091E50095E6409151
:10337000EC00842F817040FF22C08091E80080FD26
:103380001CC080918304882391F0853091F0809156
:10339000EB0085FD10C04091E4005091E50042171C
:1033A000530729F39A01915011F784E0089582E0C0
:1033B000089583E0089581E0089580E008954091A4
:1033C000E80042FFDECF08950E94521A0E945A1A66
:1033D000E0EEF0E0808181608083E8EDF0E08081C4
:1033E0008F77808319BCA7EDB0E08C918E7F8C9392
:1033F00080818F7E80831092820408950F931F93A3
:10340000CF93DF930E94521A0E945A1AC8EDD0E05F
:1034100088818F77888388818068888388818F7D81
:10342000888319BC1092830410927F041092810447
:103430001092800400EE10E0F80180818B7F808381
:1034400088818160888342E060E080E00E945E19AC
:10345000E1EEF0E080818E7F8083E2EEF0E080811B
:1034600081608083808188608083F80180818E7F85
:103470008083888180618883DF91CF911F910F9134
:103480000895E8EDF0E080818F7E8083E7EDF0E045
:1034900080818160808384E082BF81E080938204A8
:1034A0000C94FE19E8EDF0E080818E7F808310920D
:1034B000E20008951092DA001092E10008951F9240
:1034C0000F920FB60F9211242F933F934F935F9358
:1034D0006F937F938F939F93AF93BF93EF93FF93DC
:1034E0008091E10082FF0BC08091E20082FF07C063
:1034F0008091E1008B7F8093E1000E94C61C809147
:10350000DA0080FF1FC08091D80080FF1BC080912F
:10351000DA008E7F8093DA008091D90080FF0DC0A1
:1035200080E189BD82E189BD09B400FEFDCF81E063
:10353000809383040E94CE1605C019BC10928304A8
:103540000E94DC168091E10080FF19C08091E200AA
:1035500080FF15C08091E2008E7F8093E200809111
:10356000E20080618093E2008091D80080628093C5
:10357000D80019BC85E0809383040E94E0168091F6
:10358000E10084FF30C08091E20084FF2CC080E124
:1035900089BD82E189BD09B400FEFDCF8091D800CC
:1035A0008F7D8093D8008091E1008F7E8093E10031
:1035B0008091E2008F7E8093E2008091E200816042
:1035C0008093E20080917F04882311F084E007C09B
:1035D0008091E30087FD02C081E001C083E0809319
:1035E00083040E94E1168091E10083FF29C080914D
:1035F000E20083FF25C08091E100877F8093E10096
:1036000082E08093830410927F048091E1008E7F9A
:103610008093E1008091E2008E7F8093E2008091B0
:10362000E20080618093E20042E060E080E00E947E
:103630005E198091F00088608093F0000E94DF1690
:10364000FF91EF91BF91AF919F918F917F916F917A
:103650005F914F913F912F910F900FBE0F901F9050
:1036600018951F920F920FB60F9211242F933F932C
:103670004F935F936F937F938F939F93AF93BF937A
:10368000CF93DF93EF93FF93C091E900CF708091C8
:10369000EC00D82FD17080FDD0E81092E900809125
:1036A000F000877F8093F00078940E94751B109241
:1036B000E9008091F00088608093F000CD2BCF70FE
:1036C000C093E900FF91EF91DF91CF91BF91AF914E
:1036D0009F918F917F916F915F914F913F912F912A
:1036E0000F900FBE0F901F9018951F93CF93DF93ED
:1036F000CDB7DEB7AA970FB6F894DEBF0FBECDBF29
:10370000E4E8F4E088E08E0F9091F10091938E133D
:10371000FBCF0E94F7168091E80083FF1FC18091C4
:10372000840490918504492F50E04A30510508F0F7
:1037300015C1FA01EC59FF4F0C948732803881F0A3
:10374000823809F00BC1809188048F708093E90062
:103750008091EB0085FB882780F91092E90006C074
:103760008091800490918104911182609091E80091
:10377000977F9093E8008093F1001092F100C8C009
:10378000282F2D7F09F0EAC0882319F0823061F0DC
:10379000E5C080918604813009F0E0C0933009F0E3
:1037A00080E0809381042BC080918604811127C022
:1037B000809188048F7009F4D1C08093E900209132
:1037C000EB0020FF1CC0933021F48091EB0080625D
:1037D00014C09091EB0090619093EB0021E030E0F9
:1037E000A90102C0440F551F8A95E2F74093EA00F1
:1037F0001092EA008091EB0088608093EB001092B9
:10380000E9008091E800877F86C08111A7C01091F0
:1038100086041F778091E3008078812B8093E300FA
:103820008091E800877F8093E8000E94931980913F
:10383000E80080FFFCCF8091E30080688093E30084
:10384000111102C082E001C083E08093830486C02E
:103850008058823008F082C080918604909187045D
:103860008C3D53E0950779F583E08A838AE289836A
:103870004FB7F894DE01139620E03EE051E2E32FCB
:10388000F0E050935700E49120FF03C0E295EF7001
:103890003F5FEF708E2F90E0EA3010F0C79601C0C6
:1038A000C0968D939D932F5F243149F74FBF809130
:1038B000E800877F8093E8006AE270E0CE0101961D
:1038C0000E949A1814C0AE014F5F5F4F6091880448
:1038D0000E94E117BC01009709F440C09091E800F4
:1038E000977F9093E80089819A810E94FD188091CA
:1038F000E8008B778093E80031C0803879F58091BB
:10390000E800877F8093E80080917F048093F10036
:103910008091E8008E778093E8000E9493191EC082
:1039200081111CC0909186049230C0F48091E8000F
:10393000877F8093E80090937F040E949319809181
:103940007F04811106C08091E30087FD02C081E001
:1039500001C084E0809383040E94E3168091E80014
:1039600083FF0AC08091E800877F8093E800809100
:10397000EB0080628093EB00AA960FB6F894DEBF4E
:103980000FBECDBFDF91CF911F9108950895CF93C2
:10399000809183048823A1F0C091E900CF709091B9
:1039A000EC00892F817090FD80E8C82B1092E9000F
:1039B0008091E80083FD0E94751BCF70C093E900E1
:1039C000CF91089590930304809302040895E091A9
:1039D0000204F0910304309721F00190F081E02D72
:1039E000099480E00895E0910204F0910304309777
:1039F00021F00280F381E02D09940895E091020402
:103A0000F0910304309721F00480F581E02D0994B2
:103A1000089520910004309101048217930771F0FA
:103A20009093010480930004E0910204F091030458
:103A3000309721F00680F781E02D099408952091B8
:103A4000FE033091FF038217930771F09093FF03F9
:103A50008093FE03E0910204F0910304309721F07B
:103A60000084F185E02D0994089508950C94351D86
:103A70000E94BC280E947E0E0E9442290C94F62DC2
:103A80005F926F927F928F929F92AF92BF92CF92EE
:103A9000DF92EF92FF920F931F93CF93DF9300D0AB
:103AA00000D01F92CDB7DEB70E94C30E9DE0C92E95
:103AB00094E0D92E03E010E0AA24A394B12C502E58
:103AC000802F0E943E0F4C01F601729062906F01B0
:103AD0006826792661147104A1F40150110978F760
:103AE0008FEF89838A831B820E94C5288160782F8B
:103AF0009D838C8349815A816B818D810E94F01D49
:103B000038C08091620481FD0E94470F2BE030E0B5
:103B10007501022E02C0EE0CFF1C0A94E2F7C701E9
:103B200086219721892B09F129835A828E209F2093
:103B300091E0892809F490E09B830E94C528816068
:103B4000782F9D838C8349815A816B818D810E945E
:103B5000F01D000F111FF801EB5FFB4F8081918179
:103B6000E826F926F182E08204C02150310980F66E
:103B7000B4CF0E942E2B109104040E94E71C18174A
:103B8000D1F00E94E71C809304040F900F900F90D7
:103B90000F900F90DF91CF911F910F91FF90EF90B9
:103BA000DF90CF90BF90AF909F908F907F906F905D
:103BB0005F900C94680E0F900F900F900F900F90E5
:103BC000DF91CF911F910F91FF90EF90DF90CF90F9
:103BD000BF90AF909F908F907F906F905F9008956F
:103BE000CF93DF93CDB7DEB72B970FB6F894DEBF38
:103BF0000FBECDBF4F83588769877A878B87DE01D9
:103C0000119686E0FD0111928A95E9F785E0FE01A3
:103C1000379601900D928A95E1F749815A816B811F
:103C20007C818D819E810E9467242B960FB6F8942B
:103C3000DEBF0FBECDBFDF91CF910895CF93882314
:103C400009F4C2C0C82F823859F40E94E71C81FDD4
:103C5000BBC089E30E9441270E940E2889E30CC063
:103C6000833879F40E94E71C80FDAEC083E50E9492
:103C700041270E940E2883E50E948327CF910C9450
:103C80000E28843859F40E94E71C82FD9DC087E409
:103C90000E9441270E940E2887E4EECF8CEF8C0F04
:103CA000813A48F48C2F0E945E2D81118DC08C2F9B
:103CB0000E944127E3CF80E28C0F883048F4C77020
:103CC00081E001C0880FCA95EAF70E94C727D6CFC6
:103CD0008BE58C0F833078F4C53A29F0C63A31F081
:103CE00083E890E005C081E890E002C082E890E0BF
:103CF000CF910C94091D88E58C0F833108F064C0C6
:103D0000C83A39F1C93A41F1CA3A49F1CB3A51F1CD
:103D1000CC3A59F1CD3A61F1C03B69F1CE3A71F13B
:103D2000CF3A79F1C13B81F1C23B89F1C33B91F1BB
:103D3000C43B99F1C53BA1F1C63BA9F1C73BB1F129
:103D4000C83BB9F1C93BC1F1CA3BC9F180E090E081
:103D500038C082EE90E035C089EE90E032C08AEE45
:103D600090E02FC085EB90E02CC086EB90E029C05E
:103D700087EB90E026C08CEC90E023C08DEC90E0C7
:103D800020C083E891E01DC08AE891E01AC082E972
:103D900091E017C084E991E014C081E292E011C083
:103DA00083E292E00EC084E292E00BC085E292E0F2
:103DB00008C086E292E005C087E292E002C08AE293
:103DC00092E0CF910C941F1DCF910895882309F4A0
:103DD0004BC0823859F40E94E71C81FF45C089E33B
:103DE0000E9441270E940E2889E30CC0833871F499
:103DF0000E94E71C80FF38C083E50E9441270E9493
:103E00000E2883E50E9483270C940E28843859F4E9
:103E10000E94E71C82FF28C087E40E9441270E947D
:103E20000E2887E4EFCF9CEF980F913A58F390E279
:103E3000980F983050F4877091E001C0990F8A95DF
:103E4000EAF7892F0E94CD27DFCF9BE5980F9330AB
:103E500020F480E090E00C94091D885A833120F40E
:103E600080E090E00C941F1D0895882321F00E94AB
:103E7000C7270C940E280895882321F00E94CD278F
:103E80000C940E2808957F928F929F92AF92BF92CA
:103E9000CF92DF92EF92FF920F931F93CF93DF9316
:103EA0001F92CDB7DEB77C01C62E772EFC010581AF
:103EB00002950F70128111110E94E4270E943A2787
:103EC000882379F0112369F080E28C0D883048F066
:103ED00082E00E9423270E943A2791E0D82ED9261B
:103EE00001C0D12CE72DE295EF70F0E0E259FF4FD1
:103EF0000C948732872D807F072D0F70882311F057
:103F00000295007F112389F0002309F499C180E212
:103F10008C0D883020F4802F0E94C72703C0802F8B
:103F20000E94D7270E940E288BC18C2D0E94E61E6E
:103F3000002309F4C3C180E28C0D883020F4802F67
:103F40000E94CD2703C0802F0E94DD270E940E28EB
:103F5000B5C1872D807F972D9F70803211F4892FF6
:103F600003C0892F8295807FCC2021F0F1E0CF160D
:103F7000A1F01DC0112339F0002319F1013009F51A
:103F80000E94F7279BC1002319F0013009F496C164
:103F900089830E94FA27898110C1112321F00630FC
:103FA00008F08CC10EC0053008F088C106C111238D
:103FB00059F0002331F0F701958190FF41C19F70C6
:103FC00095830E94351F7AC1002309F4F6C03EC1D3
:103FD000872D86958695837090E0009719F001975C
:103FE00061F06CC1112321F08C2D972D937002C0CC
:103FF00080E090E00E94091D61C1112321F08C2D09
:10400000972D937002C080E090E00E941F1D56C162
:104010008C2D112319F00E94362A02C00E949E2A7C
:104020000E94232B4BC1872D837009F052C01111C0
:1040300045C18C2D829586958770880F880F9C2DA1
:104040009F70892E912CA12CB12C082E04C0880CB5
:10405000991CAA1CBB1C0A94D2F7C4FE14C00FE022
:1040600010E020E030E0B901A80104C0440F551F62
:10407000661F771F8A95D2F7CB01BA0160957095BC
:104080008095909503C060E070E0CB01272D2695C8
:104090002695237030E02230310569F02330310558
:1040A00089F0682979298A299B292130310571F005
:1040B0000E94AF2503C1682979298A299B290E947A
:1040C000CB25FCC00E94AF25C501B4010E949325F9
:1040D000F5C0112319F0872D817001C086958823C2
:1040E00009F4ECC08C2D829586958770880F880F17
:1040F0009C2D9F70892E912CA12CB12C082E04C0D0
:10410000880C991CAA1CBB1C0A94D2F7C4FE14C0CC
:104110000FE010E020E030E0B901A80104C0440F36
:10412000551F661F771F8A95D2F7CB01BA0160959C
:1041300070958095909503C060E070E0CB01272DCD
:10414000269526952370422F50E04230510569F0A4
:104150004330510589F0682979298A299B29413002
:10416000510571F00E948926A9C0682979298A29F8
:104170009B290E94A526A2C00E948926C501B401E0
:104180000E946D269BC08C2D90E0FC01E05EF10941
:10419000E531F10508F050C0E258FF4F0C9487322A
:1041A0000C2D0F70872D8F71112321F00E94062690
:1041B000802F07CF0E942726802F0E943C1F7EC0A1
:1041C000112341F0053008F079C0872D8F710E94CE
:1041D0004C2674C0063008F071C0F7CF112339F0B7
:1041E000872D8F710E94062669C01123C9F3872D80
:1041F0008F710E94272662C0112329F0872D8F71AD
:104200000E94F1255BC00E94E72558C0112351F0A0
:10421000172D1F71812F0E94062663E0812F0E94B7
:104220001A274CC081E00E942327023008F446C0C0
:1042300082E00E94232742C0112331F0002381F243
:104240008C2D0E941E1E3AC0002389F28C2D0E94E4
:10425000E61E34C0472D4F706C2DC7010E940B071E
:104260000E940B252BC0111129C0472D4F7050E023
:1042700042305105B9F04CF44115510581F04130FF
:104280005105E1F40E941E2E19C04330510569F01A
:104290004430510599F48C2D0E94702E0FC00E945D
:1042A000072E0CC00E943A2E09C00E944D2E06C057
:1042B000472D4F706C2DC7010E94090BDD20F9F0CE
:1042C0000E94162780FD1BC0F70112820E94102752
:1042D0000E940626C7010E948E210E9410270F907F
:1042E000DF91CF911F910F91FF90EF90DF90CF90D2
:1042F000BF90AF909F908F907F900C9427260F9047
:10430000DF91CF911F910F91FF90EF90DF90CF90B1
:10431000BF90AF909F908F907F9008950F931F93C1
:10432000CF93DF93EC01888199812B813C81232BF2
:10433000B9F09F3F11F48F3F99F0CE010E94080918
:10434000882371F0688179818A810E940C278C0111
:104350000E94C1260E948825B801CE010E94431FF9
:10436000DF91CF911F910F9108950E94E4270E9441
:10437000F4270E94B9270E940E280E94D42B0E9485
:10438000232B80E090E00E94091D80E090E00C94D7
:104390001F1D0E94D4270C94B5210E940127292FAC
:1043A00022952F7030E02C3031054CF42A30310545
:1043B0006CF42250310922303105A8F407C02C30AA
:1043C000310569F02F30310551F00DC0803F69F0A3
:1043D00018F4803E40F409C0843F29F406C093FBE2
:1043E000882780F9089580E0089581E00895CF93AB
:1043F000DF9300D000D01F92CDB7DEB70F900F90A3
:104400000F900F900F90DF91CF910895CF93DF938E
:1044100000D000D000D0CDB7DEB726960FB6F89406
:10442000DEBF0FBECDBFDF91CF9108951F93CF9315
:10443000DF93C0910D0416E080910E04C81799F027
:10444000D0E01C9FF0011D9FF00D1124E15FFB4F98
:104450004081518162817381848195810E9406220D
:104460002196C770E9CFDF91CF911F9108954091B8
:104470003F04509140046091410470914204809146
:104480004304909144040C94062280914404829544
:104490008F7009F054C080914104882309F44FC003
:1044A00080910D04A0910E0460913F04709140042E
:1044B0004091420450914304B6E08A1709F43FC08A
:1044C00090E041155105C1F17F3F11F46F3FA1F11B
:1044D000B89FF001B99FF00D1124E15FFB4F2181DE
:1044E00072132AC02081621327C02281211124C0A7
:1044F000238134812417350710F421503109241BFE
:10450000350B283C3105C0F4209144042F70206104
:104510002093440426E0289FF001299FF00D1124E8
:10452000EC5EFB4F80818F70806180838FE394E02D
:104530000E948E210C94162201968770BECF08959A
:10454000CF92DF92EF92FF920F931F93CF93DF935F
:10455000CDB7DEB762970FB6F894DEBF0FBECDBF02
:104560008C0185E0F801DE011D9601900D928A957F
:10457000E1F7D8014C9111965C91119712966C91CC
:1045800012971396CD90DC90149730913F04709160
:1045900040048091420490914304009709F46BC158
:1045A0007F3F19F43F3F09F466C1E0904104EE20DB
:1045B00009F4C0C020914404C816D90628F0F601B9
:1045C000E81BF90BCF0104C0809590958C0D9D1DC3
:1045D000FF24F394883C910578F0F12C207F09F0BA
:1045E000C6C07C2DD98AC88A89890E94F7218FE3A9
:1045F00094E00E948E21B1C0822F807F09F046C0D6
:10460000751314C0341312C0611110C02F702061D3
:10461000209344040E9437228FE394E00E948E216D
:1046200080914404D80115968C932EC0CD2819F1A1
:104630005F3F11F44F3FF9F0F62E61111CC08091DD
:104640000D0420910E0436E0821709F45AC090E060
:10465000389FF001399FF00D1124E15FFB4F71810C
:10466000571306C07081471303C07281711103C0D4
:1046700001968770E9CFF62E662309F418C1809160
:104680004404816080934404F12C11C1751308C067
:10469000341306C0611104C080914404D801C3C022
:1046A0004D875E878D859E856A8B0E94CD216A89A4
:1046B0008823E1F16623D1F120914404822F829571
:1046C0008F7090E0029774F080913F0490914004C5
:1046D00098878F831986DB86CA862C87CE0107963A
:1046E0000E948E2186E0F801AFE3B4E001900D92C4
:1046F0008A95E1F70E9445220E943722FF24F39415
:10470000D6C04D875E878D859E850E940127292F03
:1047100022952F7030E0223031050CF0BCC09F7024
:1047200009F0B6C0805E883008F4C1C0C8010E949C
:104730008E21E4CFC816D90608F453C0F601E81B51
:10474000F90BCF01883C910508F450C0F12C7C2D69
:10475000D98AC88A89890E94F721EFE3F4E086E0CC
:10476000DF011D928A95E9F70E943722A0C07513D8
:1047700014C0341312C0611110C080914404F801B8
:104780008583C8010E948E2186E0EFE3F4E0DF011B
:104790001D928A95E9F7FE2C8AC04D875E878D852C
:1047A0009E856A8B0E94CD216A89882309F4BECF39
:1047B000662309F4BBCF20914404822F82958F7029
:1047C00090E002970CF48ECF80913F0490914004CA
:1047D0009A8389831B82DD82CC822E83CE0101964F
:1047E0007FCF809590958C0D9D1DACCFF62E6623C6
:1047F00009F49CCF75132EC034132CC020914404AF
:1048000020FD1FC0822F82958F70D9F0D801159698
:104810002C9315978F3049F08F5F982F9295907F4A
:10482000822F8F70892B15968C93C8010E948E2140
:1048300086E0F801AFE3B4E001900D928A95E1F7CC
:1048400093CF86E0F801AFE3B4E001900D928A9532
:10485000E1F72DC04D875E878D859E850E94CD2115
:10486000811140CF80914404816080934404C80149
:104870000E948E211CC0662309F458CF4D875E87A5
:104880008D859E850E94CD21882309F44FCF2ACFA4
:10489000811148CF0CC0243031050CF047CF9F70F8
:1048A00009F440CFF8019581907F09F03BCF8F2D1F
:1048B00062960FB6F894DEBF0FBECDBFDF91CF91E9
:1048C0001F910F91FF90EF90DF90CF9008951F936D
:1048D000CF93DF93CDB7DEB72C970FB6F894DEBF3A
:1048E0000FBECDBF4F83588769877A878B879C8798
:1048F000CE0107960E94A022882369F08F819885B7
:104900002A853B85232BF1F19F3F09F063C08F3F40
:1049100009F060C037C086E0FE013796DE011196CF
:1049200001900D928A95E1F76F817885EA85FB8584
:10493000309741F17F3F11F46F3F21F120910E0438
:1049400030E0C90101968770992740910D0450E02D
:104950008417950709F447C069837A83FD83EC8344
:1049600096E0929FD001939FB00D1124A15FBB4FA1
:10497000FE01319601900D929A95E1F780930E0415
:104980000E94162216E080910D0490910E04891762
:10499000C1F1189FC0011124815F9B4F0E94A0228A
:1049A000882379F1E0910D041E9FF0011124E15F4D
:1049B000FB4F4081518162817381848195810E9486
:1049C000062280910D0490E00196877099278093CC
:1049D0000D04D9CF4F81588569857A858B859C8553
:1049E0000E940622CFCF0E94C92110920E0410927D
:1049F0000D04EFE3F4E086E0DF011D928A95E9F70C
:104A0000C1CF2C960FB6F894DEBF0FBECDBFDF919D
:104A1000CF911F910895EF92FF920F931F93CF9321
:104A2000DF938C01009709F46CC0F12CEE24E39421
:104A3000E8012196F8018491843740F4843008F02D
:104A400051C0813081F0823019F15BC0853709F4A3
:104A500044C0A8F19CE7980F903708F052C08F77B8
:104A60000E94E61E41C00E5F1F4FFE01C49180E20E
:104A70008C0F883048F4C7708E2D01C0880FCA95FE
:104A8000EAF70E94E72714C08C2F0E941E1E2DC03B
:104A90000E5F1F4FFE01C49180E28C0F883058F4E6
:104AA000C7708E2D01C0880FCA95EAF70E94ED27C6
:104AB0000E940E281AC08C2F0E94E61E16C00E5FA0
:104AC0001F4FFE01C491CC2381F08FE99FE0019735
:104AD000F1F700C00000C150F6CF0E5F1F4FFE017E
:104AE000F49003C00E941E1E8E018F2D882309F4AE
:104AF0009FCFEFE9FFE03197F1F700C00000815050
:104B0000F5CFDF91CF911F910F91FF90EF90089516
:104B100008956093490470934A0480934B049093E2
:104B20004C040C94B5210F931F93009149041091EC
:104B30004A0420914B0430914C04DC01CB01802BC2
:104B4000912BA22BB32B8093490490934A04A093FA
:104B50004B04B0934C041F910F910C94B5210F930B
:104B60001F930091490410914A0420914B04309105
:104B70004C04DC01CB0180239123A223B323809337
:104B8000490490934A04A0934B04B0934C041F91A2
:104B90000F910C94B5210F931F930091490410912C
:104BA0004A0420914B0430914C04DC01CB01802756
:104BB0009127A227B3278093490490934A04A09396
:104BC0004B04B0934C041F910F910C94B52110929B
:104BD00045041092460410924704109248040C9425
:104BE000B52141E050E060E070E004C0440F551F83
:104BF000661F771F8A95D2F7409345045093460469
:104C000060934704709348040C94B52141E050E050
:104C100060E070E004C0440F551F661F771F8A953F
:104C2000D2F78091450490914604A0914704B09139
:104C30004804482B592B6A2B7B2B409345045093F7
:104C4000460460934704709348040C94B52141E0F6
:104C500050E060E070E004C0440F551F661F771FEE
:104C60008A95D2F74095509560957095809145044E
:104C700090914604A0914704B091480448235923D9
:104C80006A237B2340934504509346046093470472
:104C9000709348040C94B52141E050E060E070E06E
:104CA00004C0440F551F661F771F8A95D2F7809165
:104CB000450490914604A0914704B09148044827C8
:104CC00059276A277B2740934504509346046093F5
:104CD0004704709348040C94B5210F931F930091DF
:104CE0004504109146042091470430914804DC01AA
:104CF000CB01802B912BA22BB32B80934504909357
:104D00004604A0934704B09348041F910F910C945C
:104D1000B5210F931F9300914504109146042091F3
:104D2000470430914804DC01CB0180239123A22366
:104D3000B3238093450490934604A0934704B09313
:104D400048041F910F910C94B5210F931F9300916C
:104D50004504109146042091470430914804DC0139
:104D6000CB0180279127A227B327809345049093F6
:104D70004604A0934704B09348041F910F910C94EC
:104D8000B5210895CF92DF92EF92FF920F931F9378
:104D9000CF93DF938C01C0904904D0904A04E090F7
:104DA0004B04F0904C048091450490914604A091EE
:104DB0004704B0914804C82AD92AEA2AFB2ACFE13D
:104DC000D0E0D701C6010C2E04C0B695A7959795E3
:104DD00087950A94D2F780FF06C0B8018C2F0E94F5
:104DE0008E0D019721F4219760F780E001C08C2F90
:104DF000DF91CF911F910F91FF90EF90DF90CF90B7
:104E00000895CF93DF93EC010E94C226BE010E9459
:104E10008E0DDF91CF910895CB010E940127089557
:104E200080914D04859585958595089580914D04D3
:104E30008770089598E0899F90011124262B209374
:104E40004D040C94062620914D0480958223809376
:104E50004D04982F977069F430E0482F552747FD8F
:104E600050952417350729F08595859585950C94DF
:104E70002726089590914D04977081E009F480E011
:104E8000089590918502992321F0909186029111C5
:104E900009C02091870230918802F90132969FEF74
:104EA00040E01FC0982F9695969596959F3050F5A7
:104EB000E0918702F0918802E90FF11D877021E0EF
:104EC00030E0A90102C0440F551F8A95E2F7CA01DC
:104ED0009181892B818308959F3F39F04F5F4E3038
:104EE00041F051915813F8CF0DC05111F7CF942FC5
:104EF000F5CF9F3F39F0F901E90FF11D97FDFA95C4
:104F000082830895089590918502992321F09091CC
:104F10008602911109C02091870230918802F9011F
:104F20003296205F3F4F1FC0982F96959695969585
:104F30009F30F0F4E0918702F0918802E90FF11DB3
:104F4000877021E030E0A90102C0440F551F8A9507
:104F5000E2F7CA0180959181892381830895319672
:104F6000E217F30729F090819813F9CF1082F7CF59
:104F7000089581E090E0E0918702F0918802E80FC7
:104F8000F91F1082019680319105A9F7089590913B
:104F90006104892B80936104089580959091610448
:104FA000892380936104089510926104089590917B
:104FB0006004892B8093600408958095909160042B
:104FC000892380936004089510926004089590915D
:104FD0005F04892B80935F040895809590915F040E
:104FE000892380935F04089510925F04089580934D
:104FF0004E04089510924E04089580918702909176
:105000008802FC0131969C01205F3F4F80E0919126
:1050100091118F5FE217F307D1F70895E0918702AE
:10502000F0918802809161048083E0918702F09181
:105030008802908180916004892B8083E0918702AF
:10504000F0918802908180915F04892B8083809108
:105050004E04882361F0E0918702F09188029081EC
:10506000892B80830E94FD27811110924E0480912C
:105070008702909188020C94F31C20E0009739F08D
:10508000AC0141505109842395232F5FF7CF822F24
:10509000089580918304843039F11092630420E4F0
:1050A00088E190E00FB6F894A895809360000FBE59
:1050B0002093600080E00E94390680E00E94680E24
:1050C00083B7817F846083BF83B7816083BF789417
:1050D000889583B78E7F83BF88E10FB6F89480935D
:1050E0006000109260000FBE08950895089580E05A
:1050F0000E9439060E9475280E94C30E0E947628DD
:105100000E94480F91E0811101C090E0892F08951D
:105110000E94C92180E00E9439060E94F62D0E945B
:10512000E71C0C94680E1F920F920FB60F92112479
:105130008F939F93AF93BF9380916304811113C0AA
:105140008091640490916504A0916604B091670415
:105150004196A11DB11D8093640490936504A093B2
:105160006604B0936704BF91AF919F918F910F90A8
:105170000FBE0F901F90189582E084BD93E095BDFF
:105180009AEF97BD80936E0008952FB7F8948091A1
:10519000640490916504A0916604B09167042FBFE8
:1051A0000895CF92DF92EF92FF920F931F932FB744
:1051B000F894409164045091650460916604709184
:1051C00067042FBF6A017B01EE24FF248C0120E0DD
:1051D00030E0C016D106E206F30610F44150510942
:1051E0009A01281B390BC9011F910F91FF90EF9075
:1051F000DF90CF9008951F920F920FB60F92112457
:105200008F939F93AF93BF938091640490916504B3
:10521000A0916604B09167040196A11DB11D809311
:10522000640490936504A0936604B0936704BF91EF
:10523000AF919F918F910F900FBE0F901F90189577
:105240000E94E419F8942FEF87EA91E621508040FC
:105250009040E1F700C0000087E090EBDC01809314
:105260008E0490938F04A0939004B09391049CE0DB
:1052700088E10FB6F894A895809360000FBE9093D4
:105280006000FFCF0E948129811102C00E945D2928
:105290000E948C29809362040E94992980938C0437
:1052A00087FB882780F9809386020E949029682FC7
:1052B00070E080E090E00C9489256DEE7EEF80E058
:1052C00090E00E94AD3260E082E090E00E949B326C
:1052D00060E083E090E00E949B3260E084E090E038
:1052E0000E949B3260E085E090E00E949B3260E08B
:1052F00086E090E00E949B326FEF87E090E00C9494
:105300009B3280E090E00E94953221E08D3E9E4FDE
:1053100009F020E0822F089582E090E00C948D3215
:1053200083E090E00C948D32682F83E090E00C9441
:105330009B3284E090E00C948D32682F84E090E002
:105340000C949B3286E090E00C948D32682F86E0BE
:1053500090E00C949B3287E090E00C948D32682FA3
:1053600087E090E00C949B3280916A0480FF0BC030
:1053700060918C0285E0689FB00111247595679556
:10538000759567952BC081FF09C060918C0285E0FF
:10539000689FB00111247595679520C082FF07C0F2
:1053A00060918C0285E0689FB001112417C0909134
:1053B0006B049923D1F060918B02961788F72091A6
:1053C0008C0285E0289F90011124929FA001939F59
:1053D000500D112470E0CA010E94733260387105CB
:1053E00040F46115710539F002C065E070E0862F68
:1053F00008958FE7089581E0089580916A0480FF01
:1054000008C060918A0270E07595679575956795FB
:1054100021C081FF06C060918A0270E07595679592
:1054200019C082FF04C060918A0270E010C09091A0
:105430006B049923C1F0609189029617A0F78091BF
:105440008A02899FC001112470E00E947332603883
:10545000710528F46115710521F0862F08958FE7F5
:10546000089581E0089561E070E0F4CF803F21F479
:105470000E94B429819504C0813F29F40E94B42977
:1054800080936E040895823F21F40E94B42981958F
:1054900004C0833F29F40E94B42980936D040895C9
:1054A000893F19F40E94FD2905C08A3F31F40E940A
:1054B000FD29819580936F0408958B3F21F40E940C
:1054C000FD29819504C08C3F29F40E94FD29809319
:1054D00070040895843F21F480916C04816017C0AA
:1054E000853F21F480916C04826011C0863F21F4D5
:1054F00080916C0484600BC0873F21F480916C0420
:10550000886005C0883F31F480916C04806180938D
:105510006C0408958D3F21F480916A0481600BC072
:105520008E3F21F480916A04826005C08F3F29F488
:1055300080916A04846080936A040895803F39F4FE
:1055400080916E0487FF6CC010926E0469C0813F29
:1055500029F480916E041816BCF362C090916D041A
:10556000823F29F497FF5CC010926D0459C0833FBD
:1055700019F41916CCF354C0893F41F480916F049B
:1055800018160CF04DC010926F044AC08A3F29F4DF
:1055900080916F0487FF44C0F6CF8B3F39F4809130
:1055A000700487FF3DC0109270043AC08C3F29F40C
:1055B000809170041816BCF333C0843F21F48091AD
:1055C0006C048E7F17C0853F21F480916C048D7F21
:1055D00011C0863F21F480916C048B7F0BC0873F04
:1055E00021F480916C04877F05C0883F31F480915D
:1055F0006C048F7E80936C0413C08D3F21F48091E6
:105600006A048E7F0BC08E3F21F480916A048D7FE7
:1056100005C08F3F29F480916A048B7F80936A04D0
:1056200080916D0481110EC080916E0481110AC0B9
:1056300080916F04811106C080917004811102C0B5
:1056400010926B0408958CE694E00E94FE1C0E9468
:10565000C528909369048093680408951F93CF939D
:10566000DF9380916804909169040E94D128AC0175
:1056700090916B04992321F020918D0230E006C0B7
:1056800020918E028AE0289F90011124421753072F
:1056900008F486C080916D04C0916E04D0916F04AF
:1056A00010917004811107C0C11176C0D11174C06E
:1056B000111172C075C09F3F19F09F5F90936B04EA
:1056C000181624F40E94B42980936D0480916D040F
:1056D00087FF05C00E94B429819580936D041C1634
:1056E00024F40E94B42980936E0480916E0487FF95
:1056F00005C00E94B429819580936E0460916D0469
:10570000662339F1C0916E04CC2319F1772767FD28
:105710007095872F972F0E94952F23E333E343E360
:105720005FE30E94A5300E94622F60936D046C2F8E
:10573000772767FD7095872F972F0E94952F23E37A
:1057400033E343E35FE30E94A5300E94622F60933E
:105750006E041D1624F40E94FD2980936F0480912D
:105760006F0487FF05C00E94FD29819580936F0417
:10577000111624F40E94FD29809370048091700416
:1057800087FF05C00E94FD29819580937004DF91F9
:10579000CF911F910C94232B9F3F09F08ECF96CF72
:1057A000DF91CF911F910895ECE6F4E085E0DF01F1
:1057B0001D928A95E9F710926B0410926A0408957D
:1057C000833081F128F4813059F08230D1F008958E
:1057D000853009F449C0B8F1863009F456C00895FF
:1057E00080918E02262F30E0280F311D2F3F31058A
:1057F00024F4680F60938E0208958FEF80938E02D9
:10580000089580918D02262F30E0280F311D2F3F03
:10581000310524F4680F60938D0208958FEF809313
:105820008D02089580918C02262F30E0280F311DC3
:105830002F3F310524F4680F60938C0208958FEF99
:1058400080938C02089580918B02262F30E0280FE0
:10585000311D2F3F310524F4680F60938B020895AA
:105860008FEF80938B02089580918A02262F30E07B
:10587000280F311D2F3F310524F4680F60938A02F1
:1058800008958FEF80938A02089580918902262FD0
:1058900030E0280F311D2F3F310524F4680F60934D
:1058A000890208958FEF809389020895833011F162
:1058B00028F4813049F0823091F00895853081F1EB
:1058C00020F18630C1F1089580918E02681720F48E
:1058D000861B80938E02089510928E020895809107
:1058E0008D02681720F4861B80938D020895109214
:1058F0008D02089580918C02681720F4861B809396
:105900008C02089510928C02089580918B02681782
:1059100020F4861B80938B02089510928B020895C9
:1059200080918A02681720F4861B80938A0208956A
:1059300010928A02089580918902681720F4861BCC
:105940008093890208951092890208950F931F93FE
:10595000873208F048C08E3108F08DC0803109F4DC
:1059600077C008F5873009F461C068F4863009F023
:105970009DC080916204817F8E7F8093620481E06C
:105980008093720494C08B3009F489C08E3009F082
:105990008DC08091620482FB222720F991E092273A
:1059A00090FB82F95EC0863109F479C060F48131E0
:1059B00009F07CC00E94C9219091860281E089276C
:1059C000809386026CC0893109F469C08B3109F07B
:1059D0006DC08091620481FB222720F991E092271B
:1059E00090FB81F93EC0883309F459C050F48932E4
:1059F00009F457C0853309F454C0873209F451C003
:105A000055C0833409F44DC028F48A3308F44EC0DD
:105A1000895332C0883409F049C00E94C9210E94CC
:105A2000780F0E94DC070E94202939C090916204FF
:105A3000892F8095817080FB90F929F0966098609D
:105A40009093620434C0997F977F9093620427C03B
:105A50008091620483FB222720F991E0922790FB3A
:105A600083F9809362049923D1F08091620481606C
:105A70008093620414C08D5141E050E060E070E01A
:105A80008A019B0104C0000F111F221F331F8A953A
:105A9000D2F7C901B8010E9489250E94C92181E07D
:105AA00006C061E070E080E090E0F5CF80E01F91FB
:105AB0000F91089580E0089580E00895CF93C82F56
:105AC00080917204813069F018F08230C9F184C08D
:105AD000E0918702F09188028081823209F07EC0D5
:105AE00007C0E0918702F09188028081823261F4E0
:105AF0008C2F0E945A2D811104C08C2F0E94A62C3D
:105B00001DC081E090E01AC08C2F0E945C2D811195
:105B100014C0C43179F048F4CB3079F0C03109F0C9
:105B200061C082E08093720408C0C93219F0C833A2
:105B300021F058C01092720455C081E0817054C0A9
:105B4000C93291F120F5C43179F1B0F4C73009F0D0
:105B500047C08EE180938E0282E380938D028AE0BB
:105B600080938C0284E180938B0288E080938A0288
:105B700088E28093890234C0CE51C63088F5EC2F7C
:105B8000F0E0EA5DFC4F80818093710429C0CE343F
:105B9000E9F020F4CB3421F56AE013C0C13579F087
:105BA000C235F1F461E00DC080917104882319F0D1
:105BB0001092710415C081E08093720415C061E0F9
:105BC00006C0809171040E94E02B0AC06AE08091B7
:105BD00071040E94562C04C01092720480E004C02C
:105BE00081E002C080E0AACFCF9108950E94812970
:105BF000811102C00E945D290E94A22980938D0418
:105C000080FF02C0869501C080E00C943906809127
:105C10008D04982F9695292F30E0233031054CF4D0
:105C20009F5F990F8170892B816080938D040E9402
:105C3000A62980918D0486950C94390680918D0457
:105C4000982F969591F09158990F8170892B809398
:105C50008D048E7F91E009F490E080918D0490FB9B
:105C600080F980938D040E94A62980918D048695E9
:105C70000C94390680918D04982F909590FB80F9B3
:105C800080938D040E94A62980918D0480FF02C01C
:105C9000869501C080E00C94390690918D04892F7F
:105CA00086958F5F8F779170843028F4880F892BC9
:105CB00080938D0402C090938D0480918D048E7F1B
:105CC00091E009F490E080918D0490FB80F980933D
:105CD0008D040E94A62980918D0486950C94390626
:105CE00020918D04922F96958927982F990F822FB6
:105CF0008170892B80938D048E7F91E009F490E070
:105D000080918D0490FB80F980938D040E94A629D8
:105D100080918D0486950C94390680918D0486952A
:105D200008955058BB27AA270ED0D1C1C2D130F058
:105D3000C7D120F031F49F3F11F41EF4B7C10EF427
:105D4000E095E7FB9FC1E92FD3D180F3BA17620733
:105D500073078407950718F071F49EF5EBC10EF4F4
:105D6000E0950B2EBA2FA02D0B01B90190010C016B
:105D7000CA01A0011124FF27591B99F0593F50F483
:105D8000503E68F11A16F040A22F232F342F4427DB
:105D9000585FF3CF469537952795A795F0405395D3
:105DA000C9F77EF41F16BA0B620B730B840BBAF0A3
:105DB0009150A1F0FF0FBB1F661F771F881FC2F70E
:105DC0000EC0BA0F621F731F841F48F48795779522
:105DD0006795B795F7959E3F08F0B3CF9395880FD9
:105DE00008F09927EE0F97958795089527D108F425
:105DF00081E008950CD06BC163D140F05AD130F0EE
:105E000021F45F3F19F03EC1511195C14FC170D1CE
:105E100098F39923C9F35523B1F3951B550BBB2771
:105E2000AA2762177307840738F09F5F5F4F220F1E
:105E3000331F441FAA1FA9F333D00E2E3AF0E0E817
:105E400030D091505040E695001CCAF729D0FE2F63
:105E500027D0660F771F881FBB1F261737074807F5
:105E6000AB07B0E809F0BB0B802DBF01FF279358AB
:105E70005F4F2AF09E3F510568F004C15CC15F3F4F
:105E8000ECF3983EDCF3869577956795B795F79593
:105E90009F5FC9F7880F911D9695879597F908958B
:105EA000E1E0660F771F881FBB1F62177307840727
:105EB000BA0720F0621B730B840BBA0BEE1F88F736
:105EC000E095089504D06894B11135C1089518D1B2
:105ED00088F09F5790F0B92F9927B751A0F0D1F0D3
:105EE000660F771F881F991F1AF0BA95C9F712C05D
:105EF000B13081F01FD1B1E008951CC1672F782F18
:105F00008827B85F39F0B93FCCF3869577956795C8
:105F1000B395D9F73EF490958095709561957F4F34
:105F20008F4F9F4F0895E89409C097FB3EF49095DA
:105F30008095709561957F4F8F4F9F4F9923A9F062
:105F4000F92F96E9BB279395F695879577956795F1
:105F5000B795F111F8CFFAF4BB0F11F460FF1BC035
:105F60006F5F7F4F8F4F9F4F16C0882311F096E9C8
:105F700011C0772321F09EE8872F762F05C0662376
:105F800071F096E8862F70E060E02AF09A95660F2F
:105F9000771F881FDAF7880F9695879597F90895E8
:105FA00088D018F011F08CD038F480C0C4C0E92F2C
:105FB0009FD0B0F35523C9F3E7FB6217730784073B
:105FC0009507A8F199F3E92FFF2788232AF0319745
:105FD000660F771F881FDAF7952F5527442332F075
:105FE00091505040220F331F441FD2F7BB27E91BAB
:105FF000F50B621B730B840BB109C1F222F4620F23
:10600000731F841FB11D31972AF0660F771F881FF9
:10601000BB1FEFCF915050405AF041F0882332F02F
:10602000660F771F881F91505040C1F7939530C07D
:106030008695779567959F5FD9F7F8CF990F0008F8
:10604000550FAA0BE0E8FEEF16161706E807F9074A
:10605000C0F012161306E407F50798F0621B730BE5
:10606000840B950B39F40A2661F0232B242B252B66
:1060700021F408950A2609F4A140A6958FEF811D09
:10608000811D089597F99F6780E870E060E00895AA
:106090009F3F31F0915020F4879577956795B7959C
:1060A000880F911D9695879597F908959FEF80EC3D
:1060B000089500240A94161617061806090608956E
:1060C00000240A9412161306140605060895092ED4
:1060D0000394000C11F4882352F0BB0F40F4BF2B43
:1060E00011F460FF04C06F5F7F4F8F4F9F4F089583
:1060F00057FD9058440F551F59F05F3F71F0479579
:10610000880F97FB991F61F09F3F79F0879508955D
:10611000121613061406551FF2CF4695F1DF08C07C
:10612000161617061806991FF1CF86957105610599
:1061300008940895E894BB2766277727CB0197F941
:1061400008957CDF08F48FEF08950BD0C0CFB1DF46
:1061500028F0B6DF18F0952309F094CFA7CF1124CB
:10616000EACFC6DFA0F3959FD1F3950F50E0551FFE
:10617000629FF001729FBB27F00DB11D639FAA279C
:10618000F00DB11DAA1F649F6627B00DA11D661FEB
:10619000829F2227B00DA11D621F739FB00DA11D0C
:1061A000621F839FA00D611D221F749F3327A00DC6
:1061B000611D231F849F600D211D822F762F6A2F62
:1061C00011249F5750408AF0E1F088234AF0EE0FE7
:1061D000FF1FBB1F661F771F881F91505040A9F7F4
:1061E0009E3F510570F04ECFA6CF5F3FECF3983E37
:1061F000DCF3869577956795B795F795E7959F5F5B
:10620000C1F7FE2B880F911D9695879597F90895F4
:10621000FA01EE0FFF1F30962105310599F1611546
:10622000710561F48038BFE39B0749F168949038A9
:10623000810561F08038BFEF9B0741F0992342F55B
:10624000FF3FE1053105210511F1E8940894E79538
:10625000D901AA2329F4AB2FBE2FF85FD0F310C0C9
:10626000FF5F70F4A695E0F7F73950F019F0FF3AA8
:1062700038F49F779F930CD00F9007FC90580895A7
:106280003EF014CF60E070E080E89FE308954FE7B0
:106290009F775F934F933F932F939ED02F913F9182
:1062A0004F915F9152DF05C019F40EF0EBCE42CF53
:1062B000FDCE26DFC8F39638C0F707F80F92E894B2
:1062C0002BE33AEA48EB5FE74EDF0F920F920F9213
:1062D0004DB75EB70F92C0D0E6E2F1E016D04F9115
:1062E0005F91EF91FF91E595EE1FFF1F49F0FE577B
:1062F000E0684427EE0F441FFA95E1F74195550BEE
:1063000032D00F9007FE26C00895DF93CF931F93DE
:106310000F93FF92EF92DF927B018C01689405C08E
:10632000DA2EEF011EDFFE01E894A591259135914B
:1063300045915591AEF3EF0106DDFE019701A801ED
:10634000DA9479F7DF90EF90FF900F911F91CF9142
:10635000DF9108959B01AC0160E070E080E89FE36D
:1063600049CD90CE95CECCDEE8F39923D9F3940FA6
:10637000511DBBF39150504094F059F0882332F0F6
:10638000660F771F881F91505040C1F79E3F5105FF
:1063900044F7880F911D9695879597F908955F3F6B
:1063A000ACF0983E9CF0BB27869577956795B7959E
:1063B00008F4B1609395C1F7BB0F58F711F460FF73
:1063C000E8CF6F5F7F4F8F4F9F4FE3CFB4CE0EF07C
:1063D0005FCE6CCE689456CE93DEC8F39923D1F38A
:1063E000C6F3DF93CF931F930F93FF92C92FDD273F
:1063F00088232AF02197660F771F881FDAF720E09D
:1064000030E040E85FEB9FE3883920F0803E30F0D9
:1064100021968F7787DCEEE4F1E003C083DCEBE7C5
:10642000F1E073DF8B01BE01EC01FB2E6F577109A8
:106430007595771F880B990B78DD28E132E741E3EA
:106440005FE38FDEAF2D9801AE01FF900F911F919A
:10645000CF91DF9178DC3BCEFA01DC01AA0FBB1FA4
:106460009B01AC01BF5728F42227332744275078DB
:106470001FC0B75188F4AB2F002446953795279558
:10648000011CA395D2F3002069F0220F331F441F93
:10649000B395DAF30DD045CC61307105A0E88A07D9
:1064A000B94630F49B01AC0166277727882790789E
:1064B000309621F020833183428353830895AA1BB1
:1064C000BB1B51E107C0AA1FBB1FA617B70710F0DF
:1064D000A61BB70B881F991F5A95A9F78095909511
:1064E000BC01CD01089597FB072E16F4009407D048
:1064F00077FD09D00E945F3207FC05D03EF49095ED
:1065000081959F4F0895709561957F4F0895EE0F87
:10651000FF1F0590F491E02D0994F999FECF92BDEB
:1065200081BDF89A992780B50895A8E1B0E042E0CE
:1065300050E00C94B532262FF999FECF92BD81BD63
:10654000F89A019700B4021639F01FBA20BD0FB6B1
:10655000F894FA9AF99A0FBE08950196272F0E948F
:106560009C320C949B32DC01CB01FC01F999FECFEB
:1065700006C0F2BDE1BDF89A319600B40D924150CB
:0A6580005040B8F70895F894FFCFDB
:10658A0052D02445000000410000DC4400000041D4
:10659A0052D0A4440000404100005C440000004185
:1065AA0048F17644000000415C978A4400000041AB
:1065BA001FD592440000004152D0A444000000417B
:1065CA005CFFB844000000410AA7CF440000004124
:1065DA000000DC44000000410AA7CF44000000414B
:1065EA000000DC4400000041000000000000804080
:1065FA0000005C45000040410000000000008040AF
:10660A0052D02445000040410AA7CF44000000416F
:10661A000000DC440000004100000000000080404F
:10662A0052D0244500004041000000000000804094
:10663A0000005C45000040410AA7CF440000004129
:10664A000000DC440000004100000000000080401F
:10665A0052D0244500004041000000000000804064
:10666A000AA74F45000040410AA7CF440000004155
:10667A000000DC44000000410000000000008040EF
:10668A0052D0244500000041000000000000804074
:10669A005CFF384500000041000000000000804017
:1066AA0052D02445000000410AA7CF44000000410F
:1066BA000000DC44000000410000000000008040AF
:1066CA0052D024450000804152D024450000404168
:1066DA005C970A450000004152D0A44400000041E2
:1066EA000000DC44000000415C970A450000A0411C
:1066FA00640007000CFF0000003F64EF157D165A86
:10670A00162616F21501014F042808140A321E0033
:10671A0002040507090B0C0E1011131517181A1C81
:10672A001D1F2123242628292B2D2F3032343537BB
:10673A00393B1F0F03764F5F6F7F496943790959C8
:10674A0053633149803F5D8B803FF8BF803FCAE188
:10675A00803F73ED803FCAE1803FF8BF803F5D8B89
:10676A00803F3149803F0000803FF16D7F3F75EAED
:10677A007E3F4C827E3F833F7E3F84287E3F833F1D
:10678A007E3F4C827E3F75EA7E3FF16D7F3F00007F
:10679A00803F404D3639340BE70AB10A780A0B0AB2
:1067AA00240A3D0A560A01020304050607080900DD
:00000001FF
